:020000040000FA
:02000000962840
:080008000C280C12990083166C
:10001000981C0828831208008C1E09008B138C1270
:100020001A08A0004130200203193528463020026A
:1000300003193B2857302002031941285A30200267
:100040000319472851302002031931284930200272
:1000500003194D280B178B17200805200D3005209C
:1000600009008312871007112A28831208148814A4
:10007000871407152A28831208108810871407157B
:100080002A28831287140715081488102A28831237
:1000900087140715081088142A288316FF30860055
:1000A00083120508A1000608A2000708A30008089B
:1000B000A4000930052081207E207B207820752037
:1000C00072206F206C2020300520842087208A2019
:1000D0008D20093005202A28A21F93289028221F4E
:1000E00093289028A21E93289028221E93289028B7
:1000F000A21D93289028221D93289028A21C9328A3
:100100009028221C93289028241F93289028A41F0D
:1001100093289028211E93289028231C9328902808
:100120003030052008003130052008008316FF30EC
:100130008500FF30860099308700C0308800890133
:1001400083128901831624309800403099008C1660
:0E0150008312903098000B178B171F10AE28EB
:02400E003A3F37
:00000001FF
